:020000040800F2
:100000005809002045010008A11000080910000847
:100010009D100008B1010008B72B00080000000087
:100020000000000000000000000000007D22000829
:10003000990D0008000000007D1C0008C92400087C
:100040005F0100085F0100085F0100085F01000810
:100050005F0100085F0100085F0100085F01000800
:100060005F0100085F0100085F0100085F010008F0
:100070005F0100085F0100085F0100085F010008E0
:100080005F0100085F0100085F0100085F010008D0
:100090005F0100085F0100085F0100085F010008C0
:1000A0005F0100085F0100085F0100085F010008B0
:1000B0005F0100082D2500085F0100085F010008AE
:1000C0005F0100085F0100085F0100085F01000890
:1000D0005F0100080D270008692700084D28000867
:1000E0005F0100085F0100085F0100085F01000870
:1000F0005F0100085F0100085F0100085F01000860
:100100005F0100085F0100085F0100085F0100084F
:100110005F0100085F0100085F0100085F0100083F
:100120005F0100085F0100085F0100085F0100082F
:10013000DFF80CD000F02AF800480047BD2C00087A
:10014000580900200648804706480047FEE7FEE7BA
:10015000FEE7FEE7FEE7FEE7FEE7FEE7FEE7FEE777
:10016000CD24000831010008D2B201E000F8012BD3
:10017000491EFBD270470022F6E710B513460A4627
:1001800004461946FFF7F0FF204610BD064C074D08
:1001900006E0E06840F0010394E807009847103457
:1001A000AC42F6D3FFF7C8FFF42E0008142F000866
:1001B00000BFFEE710B502460B460020002104E018
:1001C000545C0444E0B24C1CE1B29942F8DBC443F5
:1001D000E0B2441CE0B210BD2DE9F04100F02EFF6A
:1001E0003F4800780A281DD13E4800783E490978EA
:1001F000884217D13B4840783B494978884211D121
:100200003848007A3849097A88420BD13548407A13
:100210003549497A884205D13448008840F4004085
:10022000324908803148008800F40040002855D049
:10023000012002F0EFFC00202D4908704870887002
:10024000C87008712B49087048708870C8700871B0
:100250002949087048708870C8700871274908706B
:1002600048708870C870087100F0E8FE00202149CD
:1002700008701C48007948701A48407988701948FD
:100280008079C8701748C079087100201C4908702F
:100290001848407848701748807888701548C078AA
:1002A000C870144800790871012001F0C1F81148A4
:1002B000407804060F48807805040E48C07806028E
:1002C000601930440B490979471800F0B7FE00F077
:1002D000B5FE00200249087004490880BDE8F0819D
:1002E00009000020CC0100200C0000200A000020A2
:1002F0002C000020160000203400002039000020CF
:100300001B00002010B588B07F480078012838D144
:1003100000207D490870FC207C490870112048703D
:100320007B48007888707A484078C8707848807830
:1003300008717748C078487175480079887107213D
:100340007248FFF737FF7149C87100207149086092
:10035000FF22E121012001F0DFFB08236B4AA821E5
:10036000012001F09BFB012001F062F801206A49A5
:10037000C1F8A4016949087000206949088000F0AB
:100380005DFE6748008840F6B83188427BDC00F0AB
:1003900055FE604884380068002857D100F04EFEB2
:1003A0006946012001F058FB0446204601F0B4FFE5
:1003B0005CA001F0BBFF04F040004028EDD100201C
:1003C0008DF80A000721684600F0E7FC55A001F00F
:1003D000ADFF9DF801004E490978884254D19DF83F
:1003E00002004B49497888424ED19DF803004849A4
:1003F0008978884248D19DF804004549C9788842E7
:1004000042D19DF805004249097988423CD14348D0
:10041000007801281BD141480078401C3F490870F2
:1004200012203A49487007213848FFF7C3FE374980
:10043000C8710020374908600823344AA8210120E8
:1004400001F02CFB01203449C1F8A40158E0002040
:10045000324908700E21344800F09FFC31A001F0B1
:1004600065FF32480178012001F03CF810202E4948
:1004700048700E212C4801F043FF2DA001F056FFDB
:10048000012008B010BD16E00020224908601120AC
:100490001E49487007211D48FFF78CFE1B49C87193
:1004A00008230A46A821012001F0F8FA01201A4980
:1004B000C1F8A40124E00020154908704870887034
:1004C000C87008711B49087048708870C87008713E
:1004D0001949087048708870C87008711749087009
:1004E00048708870C870087130200F4948700E211C
:1004F0000D4801F005FF12A001F018FF0120C0E730
:1005000000F09CFD0020BCE73E00002041000020E0
:100510002C000020A4812142008021428100002083
:10052000200000200A000000C00300202A00002054
:100530004F4B0A00390000201B000020160000204D
:10054000333030300A00000010B588B03C480088D5
:1005500040F2DC51884268DA3A480068002861D1EC
:1005600000F06CFD6946012001F076FA044604F0C3
:100570004000402856D100208DF80A000721684627
:1005800000F00BFC30A001F0D1FE9DF8010078B91D
:100590009DF8020060B99DF8030048B900202B497E
:1005A000087048708870C8700871012008B010BDCC
:1005B0002748007807280FD10020244908709DF8AB
:1005C000000048709DF8010088709DF80200C87016
:1005D0009DF80300087123E01D480078082810D119
:1005E0009DF80100194908709DF8020048709DF8B7
:1005F000030088709DF80400C8709DF8050008711C
:100600000EE00020114908709DF8010048709DF827
:10061000020088709DF80300C8709DF804000871FE
:100620000120C3E700F00AFD08E000200749087038
:1006300048708870C87008710120B7E70020B5E7DE
:1006400032000020208121420A00000039000020F1
:100650002A00002010B500F0F1FCFE4800780828C0
:1006600029D1FD480078752825D1FB4840787028AD
:1006700021D1F948807864281DD1F748C0786128D5
:1006800019D1F5480079742815D1F34840796528C7
:1006900011D10020EF49087000BFF048006800F455
:1006A000E060EF490843001DEC490860BFF3408F4C
:1006B00000BF00BFFEE7E8480078752807D0E6488D
:1006C0000078FA2803D00020E249087010BDE14804
:1006D00000780E2800DAF9E7DE480078401EDE498F
:1006E000085CFB2800D0F1E7DB48807AA02804D121
:1006F000D8480078152800D0E8E7D64800780E28BA
:100700001ED1D5480078FA2814D1D348407BFB2865
:1007100010D1D448008840F40040D249088000201D
:10072000CC4908700E21CC4800F037FBCEA001F078
:10073000FDFD4AE00020C7490870CA49088044E02E
:10074000C448007815281ED1C3480078FA2814D16F
:10075000C148007DFB2810D1C248008840F4004009
:10076000C04908800020BB4908701521BA4800F034
:1007700014FBBDA001F0DAFD27E00020B5490870A8
:10078000B849088021E0B348007811281DD1B2484B
:100790000078FA2814D1B048007CFB2810D1B14869
:1007A000008840F40040AF4908800020A949087043
:1007B0001121A94800F0F1FAABA001F0B7FD04E067
:1007C0000020A4490870A7490880A648008800F4C2
:1007D0000040002871D000F031FC9F488079A34987
:1007E00088719D48C179A148C1719B48017A9F4891
:1007F00001729948417A9D4841729748807A9B4995
:100800008872084680799A4988719848C1799848D1
:10081000C1719648017A964801729448417A944889
:1008200041729248807A94284CD018DC732834D0D6
:100830000CDC252825D004DC21281AD022287DD1E3
:100840001BE0262821D07128F9D122E0742828D075
:1008500075282AD078282CD08228F0D12EE0A03814
:1008600009286BD2DFE800F0329CA0F5F4F3F2F136
:10087000F00000207D498872CBE100207B4988721E
:10088000C7E1002079498872C3E100207749887266
:10089000BFE1002075498872BBE10020734988726E
:1008A000B7E1002071498872B3E100206F49887276
:1008B000AFE100206D498872ABE1AEE100206B49E9
:1008C0008872A6E1002069498872A2E1002061498E
:1008D000087066488079674988716448C1796548BD
:1008E000C1716248017A634801726048417A614887
:1008F00041725E48807A5F4988725748407B5B4905
:1009000048735548817B594881735348C17B574888
:10091000C1735148017C554801744F48417C53488C
:1009200041744D48407B544908704B48807B487067
:100930004948C07B88704848007C00E068E1C87086
:100940004548407C087101204C49087000204C4902
:100950000880012000F06CFD4AA001F0E7FC04E0F3
:10096000FFF7D0FC044604B100E0F9E700BF45A062
:1009700001F0DCFC00204549087048708870C870A0
:1009800008714349087048708870C87008714149FF
:10099000087048708870C87008713449887238E1EE
:1009A00000203249887234E13948407848B93848E3
:1009B000807830B93648C07818B93548007900B920
:1009C00027E100202349087028488079324988713E
:1009D0002648C1793048C1712448017A2E480172F5
:1009E0002248417A2C4841722048807A2A498872EC
:1009F0000120C8720620087300204873244801783B
:100A000025488173224841782348C1732048817862
:100A1000214801741E48C1781F4841741C4801795F
:100A20001D488174162101F06BFC322002F0F2F8AF
:100A30001621194800F0B1F90BA001F077FC002055
:100A400013490870487029E099E0DDE0D8E0D3E070
:100A50002BE029E003000020040100200CED00E061
:100A60000000FA05040000200A000000F80200203F
:100A700094020020C00300202C0000203E00002033
:100A800020000020303030300A0000003900002003
:100A90001B000020160000205C0300208870C87036
:100AA00008715F498872B4E0B3E000205D490870C6
:100AB0005D480178012000F015FD00205B490880A9
:100AC0005BA001F033FC04E0FFF73EFD044604B1F7
:100AD00000E0F9E700BF56A001F028FC50488079FB
:100AE000554988714E48C1795348C1714C48017AC3
:100AF000514801724A48417A4F4841724848807AC9
:100B00004D4988720120C87206200873002048737E
:100B10004A48017848488173484841784648C1733B
:100B200046488178444801744448C1784248417439
:100B30004248017940488174162101F0E1FB3220DE
:100B400002F068F816213C4800F027F939A001F0BE
:100B5000EDFB00203949087048708870C870087132
:100B60003749087048708870C87008713549087036
:100B700048708870C87008712949887249E0324805
:100B8000407B29490870264880793049887124487B
:100B9000C1792E48C1712248017A2C48017220483F
:100BA000417A2A4841721E48807A28498872012079
:100BB00048700E21254801F0A3FB322002F02AF8EC
:100BC000194800782249088001F062FB00201B4987
:100BD000087048708870C8700871194908704870AA
:100BE0008870C87008711749087048708870C8709C
:100BF00008710B4988720CE000200949887208E0EE
:100C000000200749887204E000200549887200E04E
:100C100000BF00BF00200F49088000BF56E500005C
:100C2000F8020020030000202A00002032000020EB
:100C3000343434340A0000005C0300203900002002
:100C40001B000020160000200401002024040020C6
:100C50002C05002004000020FA204A4908701020CA
:100C600048700020887000214648C17001714171B0
:100C700000204449887100214248C17101724172CB
:100C800000204049C87400213E480175FB203D49C1
:100C90004875FA203C490870102048700020887080
:100CA00000213948C17001714171002036498871B5
:100CB00000213548C171017241720020324981F82A
:100CC0004B000021304880F84C10FB202E4981F861
:100CD0004D00FA202D4908701020487000208870BF
:100CE00000212A48C1700171417100202749887193
:100CF00000212648C1710172417200202349C87247
:100D0000002122480173FB2020494873FA20204922
:100D10000870102048700020887000211C48C170A5
:100D20000171417100201A49887100211848C17170
:100D30000172417200201649C874002114480175DF
:100D4000FB2013494875FA2012490870102048709A
:100D50000020887000210F48C1700171417100208E
:100D60000C49887100210B48C17101724172002049
:100D70000849C872002107480173FB2005494873E0
:100D80007047000094020020F80200202404002094
:100D90005C030020C003002070472DE9F0410446A9
:100DA0000E460DE02578281100F030F9074601F0D5
:100DB000B3FA284600F02AF9074601F0ADFA641CA0
:100DC0003000A6F10101CEB2ECD1BDE8F081000007
:100DD00030B5044604254FF4302000F06FF8054686
:100DE000042D17D10C48006940F002000A4908613F
:100DF00008464461006940F0400008614FF430202B
:100E000000F05CF805460448006941F6FD710840B1
:100E100001490861284630BD0020024004200B49EA
:100E2000C96801F0010109B101200EE00749C96854
:100E300001F0040109B1022007E00449C96801F08A
:100E4000100109B1032000E0042070470020024097
:100E50000348006940F080000149086170470000C4
:100E60000020024070B504460D460426F00200F052
:100E700025F80646042E11D10948006940F001000A
:100E8000074908612580F00200F018F8064604487A
:100E9000006941F6FE71084001490861304670BDA5
:100EA00000200240024803494860034848607047F8
:100EB0002301674500200240AB89EFCD00B5024613
:100EC0000423FFF7ABFF034603E0FFF7A7FF03464A
:100ED000521E012B01D1002AF7D102B90523184671
:100EE00000BD2DE9F0410246002500260020002328
:100EF0000024002791F803C00CF00F0591F803C0FF
:100F00000CF0100CBCF1000F03D091F802C04CEAB9
:100F1000050591F800C0BCF1000F31D01468002025
:100F20002BE04FF0010C0CFA00F3B1F800C00CEA12
:100F300003069E4220D183004FF00F0C0CFA03F7FA
:100F4000BC4305FA03FC4CEA040491F803C0BCF16D
:100F5000280F06D14FF0010C0CFA00FCC2F814C0A7
:100F60000AE091F803C0BCF1480F05D14FF0010C25
:100F70000CFA00FCC2F810C0401C0828D1D3146041
:100F8000B1F800C0BCF1FF0F34DD546800202EE042
:100F900000F1080C4FF0010808FA0CF3B1F800C09A
:100FA0000CEA03069E4221D183004FF00F0C0CFA8D
:100FB00003F7BC4305FA03FC4CEA040491F803C0B0
:100FC000BCF1280F05D100F1080C08FA0CF8C2F8A2
:100FD000148091F803C0BCF1480F07D100F1080C50
:100FE0004FF0010808FA0CF8C2F81080401C0828DD
:100FF000CED35460BDE8F081416170470161704714
:1010000001460A8890B2704700BFFEE70146002003
:1010100001F00F02092A04DC01F00F0202F1300096
:1010200003E001F00F023732D0B270474CF6CC40EB
:1010300001490860704700000030004010B500F022
:1010400013F810BD70B505460C4645F2555000F03A
:101050001FF8284600F010F8204600F013F800F0C2
:1010600003F8FFF7E3FF70BD4AF6AA2001490860C4
:1010700070470000003000400149486070470000A0
:101080000030004001498860704700000030004097
:1010900001490860704700000030004000BFFEE7D3
:1010A000704700007CB5054612A103C9CDE90001D7
:1010B0000821284601F0BAF805236A46302128465F
:1010C00000F0ECFC05236A461021284600F056FC8F
:1010D000002406E01DF80400A52800D003E0601CF1
:1010E000C4B2052CF6DB00BF052C01D001207CBD6D
:1010F0000020FCE7A5A5A5A5A500000008B50121D5
:101100001C2000F0CDFD4020ADF8000010208DF82F
:10111000030003208DF8020069463048FFF7E1FE26
:1011200040212E48FFF76AFF1020ADF80000694605
:101130002B48FFF7D6FE10212948FFF75FFF01205B
:10114000ADF8000048208DF8030003208DF8020060
:1011500069462348FFF7C5FE4FF40070ADF8000064
:1011600010208DF8030003208DF8020069461B480B
:10117000FFF7B7FE4FF400711848FFF73FFF4FF439
:101180008050ADF8000069461448FFF7AAFE4FF4FE
:1011900080511248FFF732FF4FF48070ADF8000025
:1011A00048208DF8030003208DF8020069460B48A3
:1011B000FFF797FE00F068FF00F024FF00200949C8
:1011C000086001200849C1F89001002005490C3150
:1011D000086001200549C1F8B00108BD000C0140BC
:1011E00000080140988121420000214200802142F4
:1011F00010B5044602222321204600F08DFC052371
:101200001E4A2A21204600F049FC05231B4A3021B2
:10121000204600F043FC3F222121204600F07CFCC8
:1012200001222221204600F077FC1A2225212046A7
:1012300000F072FC24222621204600F06DFC0F22D3
:101240002021204600F068FC0A223121204600F0CF
:1012500063FC01223D21204600F05EFC00223C217F
:10126000204600F059FC70222721204600F054FC53
:10127000FF22E221204600F04FFC10BDD92E0008CD
:1012800010B5044602222321204600F045FC052328
:101290001E4A2A21204600F001FC05231B4A30216A
:1012A000204600F0FBFB3F222121204600F034FCC9
:1012B00001222221204600F02FFC12222521204667
:1012C00000F02AFC04222621204600F025FC0F22F3
:1012D0002021204600F020FC0A223121204600F087
:1012E0001BFC01223D21204600F016FC00223C217F
:1012F000204600F011FC70222721204600F00CFC53
:10130000FF22E221204600F007FC10BDCA2E000893
:1013100010B5044602222321204600F0FDFB0523E0
:101320001E4A2A21204600F0B9FB05231B4A302122
:10133000204600F0B3FB30222121204600F0ECFBD8
:1013400001222221204600F0E7FB1222252120461F
:1013500000F0E2FB21222621204600F0DDFB0F22D7
:101360002021204600F0D8FB0A223121204600F03F
:10137000D3FB00223D21204600F0CEFB01223C2180
:10138000204600F0C9FB70222721204600F0C4FB54
:10139000FF22E221204600F0BFFB10BDBB2E00085B
:1013A00010B5044601222321204600F0B5FB052399
:1013B0001E4A2A21204600F071FB05231B4A3021DA
:1013C000204600F06BFB30222121204600F0A4FBD8
:1013D00001222221204600F09FFB192225212046D0
:1013E00000F09AFB04222621204600F095FB0F22F4
:1013F0002021204600F090FB06223121204600F0FB
:101400008BFB01223D21204600F086FB00223C217F
:10141000204600F081FB70222721204600F07CFB53
:10142000FF22E221204600F077FB10BDE82E0008E5
:1014300010B504461CB900202749086003E00020CD
:1014400025490C31086001222321204600F064FB6D
:101450000323224A2A21204600F020FB0323204AAE
:101460003021204600F01AFB01222121204600F005
:1014700053FB01222221204600F04EFB2A22252187
:10148000204600F049FB04222621204600F044FBC0
:101490000F222021204600F03FFB06223D2120465E
:1014A00000F03AFB01223C21204600F035FB70227F
:1014B0002721204600F030FBFF22E221204600F0E9
:1014C0002BFB1CB901200449086003E001200249FC
:1014D0000C31086010BD000098812142B12E000837
:1014E000AC2E000870B504460D461CB900202649F4
:1014F000086003E0002024490C3108600C2D37D22D
:10150000DFE805F0060A0E12161A1E22262A2E32CF
:101510002046FFF7FDFE2BE0204600F057F927E0BC
:10152000204600F0E3F923E02046FFF7A9FE1FE084
:10153000204600F003F91BE0204600F06FF817E0AA
:101540002046FFF755FE13E0204600F0AFF80FE00D
:10155000204600F083F90BE02046FFF721FF07E06B
:10156000204600F013F803E02046FFF7D1FE00BF4D
:1015700000BF1CB901200449086003E001200249B2
:101580000C31086070BD00009881214210B50446FE
:1015900002222321204600F0BFFA04231E4A2A21FA
:1015A000204600F07BFA04231B4A3021204600F03D
:1015B00075FA30222121204600F0AEFA01222221C4
:1015C000204600F0A9FA20222521204600F0A4FAA6
:1015D00024222621204600F09FFA0F2220212046B7
:1015E00000F09AFA08223121204600F095FA0122F3
:1015F0003D21204600F090FA00223C21204600F0D8
:101600008BFA70222721204600F086FAFF22E22181
:10161000204600F081FA10BDED2E000810B50446FA
:1016200002222321204600F077FA05231E4A2A21B0
:10163000204600F033FA05231B4A3021204600F0F3
:101640002DFA30222121204600F066FA01222221C3
:10165000204600F061FA12222521204600F05CFAB3
:1016600024222621204600F057FA0F22202120466E
:1016700000F052FA0A223121204600F04DFA0122F0
:101680003D21204600F048FA00223C21204600F08F
:1016900043FA70222721204600F03EFAFF22E22181
:1016A000204600F039FA10BDD42E000810B50446CB
:1016B00001222321204600F02FFA05231E4A2A2169
:1016C000204600F0EBF905231B4A3021204600F0AC
:1016D000E5F930222121204600F01EFA01222221C4
:1016E000204600F019FA10222521204600F014FAB5
:1016F00004222621204600F00FFA0F222021204646
:1017000000F00AFA06223121204600F005FA0122F3
:101710003D21204600F000FA00223C21204600F046
:10172000FBF970222721204600F0F6F9FF22E22182
:10173000204600F0F1F910BDDE2E000810B5044679
:1017400002222321204600F0E7F905231E4A2A2120
:10175000204600F0A3F905231B4A3021204600F063
:101760009DF930222121204600F0D6F901222221C4
:10177000204600F0D1F912222521204600F0CCF9B4
:1017800024222621204600F0C7F90F2220212046DE
:1017900000F0C2F908223121204600F0BDF90122F3
:1017A0003D21204600F0B8F900223C21204600F0FF
:1017B000B3F970222721204600F0AEF9FF22E22182
:1017C000204600F0A9F910BDCF2E000810B5044640
:1017D00003222321204600F09FF905231E4A2A21D7
:1017E000204600F05BF905231B4A3021204600F01B
:1017F00055F93F222121204600F08EF93F22222177
:10180000204600F089F928222521204600F084F99D
:1018100004222621204600F07FF90B2220212046B9
:1018200000F07AF90A223121204600F075F90122F0
:101830003D21204600F070F900223C21204600F0B6
:101840006BF970222721204600F066F9FF22E22181
:10185000204600F061F910BDC02E000810B5044606
:1018600001222321204600F057F903231E4A2A2192
:10187000204600F013F903231B4A3021204600F0D4
:101880000DF930222121204600F046F901222221C3
:10189000204600F041F92A222521204600F03CF99B
:1018A00004222621204600F037F90F22202120466D
:1018B00000F032F907223121204600F02DF90022F4
:1018C0003D21204600F028F901223C21204600F06D
:1018D00023F970222721204600F01EF9FF22E22181
:1018E000204600F019F910BDE32E000810B504469B
:1018F00003222321204600F00FF905231E4A2A2146
:10190000204600F0CBF805231B4A3021204600F08A
:10191000C5F830222121204600F0FEF801222221C4
:10192000204600F0F9F810222521204600F0F4F8B6
:1019300004222621204600F0EFF80F222021204625
:1019400000F0EAF80A223121204600F0E5F80122F1
:101950003D21204600F0E0F800223C21204600F026
:10196000DBF870222721204600F0D6F8FF22E22182
:10197000204600F0D1F810BDC52E00082DE9F04733
:101980008046894615461E46B8F1000F16D1002044
:10199000174908604946404600F0F4FB074600241A
:1019A00006E0FF21404600F0EDFB2855601CC4B264
:1019B000B442F6DB01200E49086015E000200D4915
:1019C00008604946404600F0DDFB0746002406E07B
:1019D000FF21404600F0D6FB2855601CC4B2B4423B
:1019E000F6DB0120034908603846BDE8F0870000B7
:1019F00090012142B081214270B505460E4685B95D
:101A00000020114908603146284600F0BBFBFF2149
:101A1000284600F0B7FB044601200C49C1F89001AC
:101A20000FE000200A4908603146284600F0AAFB72
:101A3000FF21284600F0A6FB044601200549C1F815
:101A4000B001204670BD00009001214200002142FB
:101A5000B08121420080214270B506460D4610211A
:101A6000304600F0E3FB07213046FFF7C5FF044690
:101A700022462721304600F04FF804F0400050B1D4
:101A80000A232A4661213046FFF778FFFF22E22130
:101A9000304600F041F8204670BD00002DE9F047C7
:101AA0008046894615461E46B8F1000F16D1002023
:101AB000174908604946404600F064FB0746002489
:101AC00006E015F8011B404600F05CFB601CC4B248
:101AD000B442F6DB01200E49086015E000200D49F4
:101AE00008604946404600F04DFB0746002406E0EA
:101AF00015F8011B404600F045FB601CC4B2B4421F
:101B0000F6DB0120034908603846BDE8F087000095
:101B100090012142B08121422DE9F04104460E4658
:101B2000154684B90020114908603146204600F06E
:101B300029FB07462946204600F024FB01200C49DA
:101B4000C1F890010FE000200A49086031462046A4
:101B500000F018FB07462946204600F013FB012041
:101B60000549C1F8B0013846BDE8F0819001214235
:101B700000002142B08121420080214208B54FF48B
:101B8000C06000F071F826208DF8000001208DF86B
:101B9000010002208DF8020001208DF80300684644
:101BA00000F02AF827208DF8000001208DF80100B0
:101BB0008DF802008DF80300684600F01DF825201E
:101BC0008DF8000000208DF8010001208DF8020042
:101BD0008DF80300684600F00FF81D208DF8000016
:101BE00000208DF801008DF8020001208DF803001F
:101BF000684600F001F808BD70B5002100230F22EF
:101C0000C47804B3154C246804F4E064C4F5E064BB
:101C1000210AC1F10403CA40447804FA03F184782C
:101C20001440214309010E4C0678A155047804F0B4
:101C30001F050124AC4005786D11AD0005F1E025CC
:101C4000C5F8004109E0047804F01F050124AC4008
:101C5000044D0678761145F8264070BD0CED00E085
:101C600000E400E080E100E002490143024A116023
:101C7000704700000000FA050CED00E0704700001E
:101C800029B1064AD2690243044BDA6104E0034AEF
:101C9000D2698243014BDA617047000000100240B4
:101CA00029B1064A92690243044B9A6104E0034A4F
:101CB00092698243014B9A61704700000010024014
:101CC00010B500F033F84FF4803000F0F1F800F078
:101CD0004DF90446012C1ED1002000F0DDF8002053
:101CE00000F018F9A00200F009F94FF4E011200407
:101CF00000F022F9012000F019F900BF392000F0AE
:101D0000A5F80028FAD0022000F024F900BF00F066
:101D1000BBF80828FBD1012144F20D00FFF7C0FFFA
:101D200001210220FFF7ACFF10BD00000F48006842
:101D300040F001000D490860084640680C49084021
:101D40000A494860084600680A490840074908608F
:101D50000846006820F4802008600846406820F4A7
:101D6000FE0048604FF41F0088607047001002407A
:101D70000000FFF8FFFFF6FE30B50021002200242E
:101D800000232D4D6D6805F00C0121B1042905D00B
:101D9000082923D105E0294D056022E0274D056083
:101DA0001FE0254D6D6805F47012234D6D6805F434
:101DB0008034022505EB92421CB9214D5543056044
:101DC0000BE01D4D6D6805F400351DB11C4D5543EC
:101DD000056002E0194D5543056002E0174D0560AE
:101DE00000BF00BF144D6D6805F0F0010909154DE5
:101DF0006B5C0568DD4045600F4D6D6805F4E06182
:101E0000090A104D6B5C4568DD4085600A4D6D68C0
:101E100005F46051C90A0B4D6B5C4568DD40C56037
:101E2000054D6D6805F44041890B074D6B5CC56835
:101E3000B5FBF3F5056130BD0010024000127A00D9
:101E400000093D00880000209800002010B50146E0
:101E50000022002300204A11012A02D1094C2368E4
:101E600006E0022A02D1074C236A01E0054C636AAE
:101E700001F01F02012494401C400CB1012000E03D
:101E8000002010BD001002400248406800F00C0025
:101E9000704700000010024001460020034A5068CD
:101EA00020F0F0000843506070470000001002402E
:101EB0001149096821F480310F4A116011460968FF
:101EC00021F480211160B0F5803F03D0B0F5802F60
:101ED0000ED106E00849096841F48031064A1160D4
:101EE00007E00549096841F4A021034A116000E0B8
:101EF00000BF00BF704700000010024001460020F4
:101F0000034A506820F4E0600843506070470000C6
:101F10000010024001460020034A506820F460503F
:101F200040EAC10050607047001002400149086655
:101F3000704700000000424202460020044B5868EF
:101F400020F47C1042EA01031843014B58607047AB
:101F50000010024001460020034A506820F00300B0
:101F600008435060704700000010024038B5002060
:101F700000900024002500BF3120FFF767FF0546D1
:101F80000098401C00900098B0F5A06F01D0002D83
:101F9000F2D03120FFF75AFF08B1012400E00024FD
:101FA000204638BD10B586B00024142101A8FEF7E4
:101FB000E2F80A2201A9084800F012F800BF07E081
:101FC00001A810F81400054A02F81400601CC4B2FD
:101FD0000A2CF5DB06B010BD000003084005002008
:101FE00070B504460D461646002300BF07E02046A4
:101FF000FFF706F825F81300A41C581CC3B2B3421F
:10200000F5DB70BD00B587B0012141F20500FFF797
:1020100047FEE020ADF8180018208DF81B000320C3
:102020008DF81A0006A91648FEF75BFFE021144858
:10203000FEF7E4FF0020ADF804004FF48270ADF825
:1020400006000020ADF80800ADF80A00ADF80C005D
:102050004FF40070ADF80E001820ADF8100000200D
:10206000ADF812000720ADF8140001A9054800F0F2
:102070006BF80121034800F04DF807B000BD0000E7
:10208000000801400030014000B587B001218803FD
:10209000FFF7F6FD01210920FFF702FE4FF4604033
:1020A000ADF8180018208DF81B0003208DF81A00D9
:1020B00006A91648FEF715FF4FF460411348FEF7D6
:1020C0009DFF0020ADF804004FF48270ADF80600CB
:1020D0000020ADF80800ADF80A00ADF80C004FF490
:1020E0000070ADF80E001820ADF810000020ADF81B
:1020F00012000720ADF8140001A9054800F024F8EB
:102100000121034800F006F807B000BD000C0140B3
:102110000038004021B1028842F04002028004E011
:1021200002884FF6BF731A400280704702460020B3
:1021300013890B400BB1012000E0002070470146DD
:10214000888970478181704710B50022028802F4A7
:1021500041520B884C8823438C882343CC882343EB
:102160000C8923434C8923438C892343CC89234303
:102170001A430280838B4FF2FF74234083830B8AC0
:10218000038210BD2DE9F04106460F4626BB06E04E
:10219000601CC4B2C82C02DB0020BDE8F081022123
:1021A0002048FFF7C3FF0028F2D039461D48FFF74B
:1021B000C9FF002405E0601CC4B2C82C01DB00206C
:1021C000EBE701211748FFF7B1FF0028F3D01548CE
:1021D000FFF7B5FFC5B222E005E0601CC4B2C82C11
:1021E00001DB0020D9E702210F48FFF79FFF0028FD
:1021F000F3D039460C48FFF7A5FF002405E0601C2A
:10220000C4B2C82C01DB0020C7E701210648FFF754
:102210008DFF0028F3D00448FFF791FFC5B2284690
:10222000BBE70000003001400038004070B50546B3
:102230000C467DB90F4800884FF6C77108400D491C
:102240000880084600882043088001210A48FFF7DB
:1022500061FF0EE0084800884FF6C7710840064944
:102260000880084600882043088001210248FFF7C3
:1022700051FF70BD0030014000380040704770B51C
:1022800004460D4629462046FEF7ECFD70BD0000D1
:1022900010B586B00024142101A8FDF76CFF00BF23
:1022A00007E00B4830F8140001A921F81400601C65
:1022B000C4B20A2CF5DB074800F0FEF80A2201A997
:1022C000044800F009F800F078FC06B010BD0000EA
:1022D0002C050020000003082DE9F04105460F46BB
:1022E0001646002400BF07E037F814102846FFF711
:1022F000C6FFAD1C601CC4B2B442F5DBBDE8F08182
:1023000070B504460D46034A2946204600F028F8D9
:1023100070BD00000038014010B504460249204657
:1023200000F00EF810BD00000044004010B5044657
:102330000249204600F02DF810BD00000044004086
:1023400070B504460D4600BF8021284600F062FBB0
:102350000028F9D02146284600F029FC012070BD54
:102360002DE9F04104460D46164614B90120BDE89A
:10237000F0810AE014F8017B31463846FFF7E0FFB0
:1023800008B90020F3E7681E85B2002DF2D10120C4
:10239000EDE770B504460E460CB9012070BD11E0A2
:1023A00014F8015B0A2D06D131460D20FFF7C8FF56
:1023B00008B90020F2E731462846FFF7C1FF08B907
:1023C0000020EBE720780028EAD10120E6E710B5ED
:1023D00000F002F810BD00000CB500200190009044
:1023E0003348006840F480303149086000BF30480D
:1023F000006800F4003000900198401C01900098A3
:1024000018B90198B0F5A06FF1D12948006800F41F
:10241000003010B10120009001E0002000900098F1
:10242000012843D12348006840F01000214908608A
:102430000846006820F0030008600846006840F085
:10244000020008601A484068194948600846406818
:1024500048600846406840F480604860084640682C
:1024600020F47C1048600846406840F4E81048605A
:102470000846006840F08070086000BF0C480068A3
:1024800000F000700028F9D00948406820F00300EF
:10249000074948600846406840F00200486000BFB5
:1024A0000348406800F00C000828F9D10CBD00007A
:1024B000001002400020024010B50446FEF7F2FC76
:1024C0002046FEF785FC10BD7047000010B513488C
:1024D000006840F001001149086008464068104952
:1024E00008400E494860084600680E4908400B49FC
:1024F00008600846006820F48020086008464068AC
:1025000020F4FE0048604FF41F008860FFF75FFF73
:102510004FF000600449086010BD00000010024048
:102520000000FFF8FFFFF6FE08ED00E010B5012106
:10253000204800F07EF800283AD001211D4800F024
:1025400069F81D480088401C1B4908801B4800880A
:10255000401C1A4908801A480088401C1849088005
:1025600018480078C0B14FF400711748FEF746FDD7
:1025700016480088401C1549088008460088B0F5B8
:10258000C87F09DB4FF400710F48FEF735FD0020CE
:102590000E4908800B4908700948008841F28831CB
:1025A000884202D1002006490880012008490870AD
:1025B00010BD000000040040200000203200002078
:1025C00022000020250000200010014026000020ED
:1025D000240000203EB505460C4601210220FFF7ED
:1025E0004FFBADF80450ADF800400020ADF80600F8
:1025F000ADF802006946064800F036F8012211469F
:10260000034800F027F80121014800F006F83EBD1C
:1026100000040040CA430282704721B1028842F0A0
:102620000102028004E002884FF6FE731A40028025
:10263000704730B50246002000230024158A05EAC1
:102640000103958905EA010413B10CB1012000E0F2
:10265000002030BD1AB183890B43838102E0838956
:102660008B43838170470000002202881D4B9842F3
:102670000ED01D4B98420BD0B0F1804F08D01B4BB1
:10268000984205D01A4B984202D01A4B984204D176
:102690004FF68F731A404B881A43174B984207D056
:1026A000164B984204D04FF6FF431A40CB881A438A
:1026B00002808B8883850B8803850A4B98420BD058
:1026C000094B984208D00E4B984205D00D4B9842CA
:1026D00002D00D4B984201D10B7A038601238382ED
:1026E00070470000002C014000340140000400400D
:1026F00000080040000C00400010004000140040A2
:1027000000400140004401400048014010B540F243
:102710002551124800F08BF988B140F225510F483D
:1027200000F0CFF80D4800F03DFAC4B20C480D4956
:10273000097844540B480078401C0A490870082165
:10274000064800F067F9012806D10821034800F087
:10275000AFF8024800F026FA10BD00000038014032
:10276000040100200300002010B540F2255112485A
:1027700000F05DF988B140F225510F4800F0A1F852
:102780000D4800F00FFAC4B20C480D4909784454C2
:102790000B480078401C0A4908700821064800F0E0
:1027A00039F9012806D10821034800F081F80248D0
:1027B00000F0F8F910BD000000440040EC040020D7
:1027C0008500002010B586B0044601210520FFF7E2
:1027D00067FA01214804FFF753FA0420ADF814000A
:1027E00003208DF8160018208DF8170005A915484C
:1027F000FEF777FB0820ADF8140004208DF81700D1
:1028000005A91048FEF76DFB01940020ADF8080003
:10281000ADF80A00ADF80C00ADF810000C20ADF8D2
:102820000E0001A9084800F051F9012240F225519B
:10283000054800F026F90121034800F051F806B0E0
:1028400010BD0000000801400044004010B540F2F7
:102850002551144800F0EBF8B0B140F22551114871
:1028600000F02FF80F4800F09DF9C4B20E480F4950
:10287000097844540D480078401C0C4908700846FB
:10288000007800F00F0008700821064800F0C2F838
:10289000012806D10821034800F00AF8014800F099
:1028A00081F910BD00480040CC0100200900002043
:1028B00001F40072B2F5007F00D100BFCA4302806C
:1028C000704710B50022002340F66A14A14200D1DF
:1028D00000BF0A1201249440A3B2DC43048010BD5F
:1028E00021B1828942F40052828104E082894DF64E
:1028F000FF731A408281704700B585B0012144F210
:102900000400FFF7CDF94FF40070ADF8000003208C
:102910008DF8020018208DF8030069463948FEF74B
:10292000E0FA4FF48060ADF8000004208DF8030059
:1029300069463448FEF7D5FA4FF41640019000205E
:10294000ADF80800ADF80A00ADF80C00ADF81000C5
:102950000C20ADF80E0001A92B4800F0B7F80122B9
:1029600040F22551284800F08CF801212648FFF755
:10297000B7FF01218804FFF783F901210820FFF741
:102980008FF94FF48060ADF8000003208DF802004D
:1029900018208DF8030069461C48FEF7A2FA4FF490
:1029A0000060ADF8000004208DF803006946174868
:1029B000FEF797FA4FF4965001900020ADF808000A
:1029C000ADF80A00ADF80C00ADF810000C20ADF821
:1029D0000E0001A90E4800F079F801A90C4800F09A
:1029E00075F8012240F22551094800F04AF801210A
:1029F0000748FFF775FF40210348FFF759FF05B06F
:102A000000BD00000008014000380140000C0140FA
:102A10000048004002460020B1F5007F00D100BF11
:102A200013880B400BB1012000E00020704770B507
:102A30000246002400230025002040F66A16B14219
:102A400000D100BFC1F3421501F01F03012606FAB1
:102A500003F3012D02D19689334006E0022D02D105
:102A6000168A334001E0968A33400C12012606FA9A
:102A700004F41688344013B10CB1012000E00020AA
:102A800070BDF0B50346002400260025002040F666
:102A90006A17B94200D100BF1846C1F3421401F0D1
:102AA0001F06012707FA06F5012C01D10C3004E0BE
:102AB000022C01D1103000E014301AB107682F4306
:102AC000076002E00768AF430760F0BD2DE9F047FB
:102AD00086B005460E460024A24600BFA146002748
:102AE000B08900B100BF2F462C8A4CF6FF7004401D
:102AF000F08804432C82AC894EF6F3100440B08871
:102B000031890843718908430443AC81AC8A4FF68C
:102B1000FF400440B0890443AC8201A8FFF72CF9C0
:102B20001F48874202D1DDF810A001E0DDF80CA0BB
:102B3000A88900F4004040B10AEBCA0000EB0A107B
:102B400031684900B0FBF1F807E00AEBCA0000EB7E
:102B50000A1031688900B0FBF1F86420B8FBF0F08E
:102B600004012009642101FB1089A88900F40040B8
:102B700040B1322000EBC900B0FBF1F000F00700DB
:102B8000044308E0322000EB09106421B0FBF1F0AF
:102B900000F00F0004432C8106B0BDE8F087000070
:102BA0000038014001468888C0F308007047C1F32F
:102BB00008028280704700BFFEE710B5FEF748F9B3
:102BC00010BD0000014A024900F013B8412C000872
:102BD0009C00002002E008C8121F08C1002AFAD198
:102BE00070477047002001E001C1121F002AFBD18D
:102BF00070472DE9F04116460F460446002503E0D4
:102C00003946B047641C6D1C20780028F8D128464E
:102C1000BDE8F08110B502460BE0C82007E01221A4
:102C200001E04B1E99B20029FBDC431E98B200283C
:102C3000F5DC1300A2F10104A2B2EED110BD000038
:102C400070B504460D46E0B20549088000BF40213A
:102C50000348001FFFF7DEFE0028F8D0204670BDB5
:102C60000438014008B501211020FFF719F80120B0
:102C7000ADF8000010208DF8030003208DF802004D
:102C800069460D48FEF72DF901210B48FEF7B6F90C
:102C90004FF40070ADF8000010208DF80300032001
:102CA0008DF8020069460448FEF71BF94FF40071E5
:102CB0000148FEF7A1F908BD00100140FFF700F838
:102CC000FEF75CFF40F271210420FEF7BBF9FEF72E
:102CD000B5F941F61F410920FFF77CFCFFF7C2FF61
:102CE000FFF70AFE4FF4E130FFF76CFDFEF706FA3E
:102CF000FEF7A4F902E039A0FFF764FF0120FEF718
:102D0000D1F90028F7D1FDF7A7FFFEF797F937486B
:102D10000068C0433649C1F88001C820FFF77AFF38
:102D20003348D0F88001C0433149C1F88001062101
:102D300030A0FEF732F831A0FFF7F8FAFEF77EF97F
:102D40002FA0FFF73FFF0120FEF772FBFFF72AF9E4
:102D50003248007832490870084600780B2833D290
:102D6000DFE800F0060A0E12161A1E22262A2E008E
:102D70002CA0FFF727FF27E02DA0FFF723FF23E07C
:102D80002EA0FFF71FFF1FE02FA0FFF71BFF1BE088
:102D900030A0FFF717FF17E031A0FFF713FF13E094
:102DA00033A0FFF70FFF0FE034A0FFF70BFF0BE09E
:102DB00035A0FFF707FF07E036A0FFF703FF03E0AA
:102DC00037A0FFF7FFFE00BF00BF3220FFF722FF52
:102DD00003E0FDF701FAFDF73DFCFAE754686520D2
:102DE000322E3447204572726F72210080012242D8
:102DF0000000224231323334353600000A00000030
:102E00000A5043B6D4C2EBC8EDBCFECDA8D3C3B0C4
:102E1000E6B1BE56312E370A000000004005002002
:102E20002A000020BDADCEF7D0ADD2E90D0A0000DA
:102E3000CCECB2A8D0ADD2E90D0A0000D4C6C4CF04
:102E4000D0ADD2E90D0A0000B9F3D6DDD0ADD2E99C
:102E50000D0A0000CBC4B4A8D0ADD2E90D0A000021
:102E6000C4DAC3C9B9C5D0ADD2E90D0A000000006B
:102E7000B0B2BBD5D0ADD2E90D0A0000C9BDCEF7C6
:102E8000D0ADD2E90D0A000056434F4DB2E2CAD48C
:102E90000D0A0000C1C9C4FEB5E7D0C50D0A000087
:102EA000C1C9C4FED2C6B6AF0D0A0000344310102B
:102EB00001344310100133200D547933200D54791F
:102EC000344310100101101043343223ABBA0134E3
:102ED00012BBAA0134128675014656431000346EA7
:102EE0004610013443101001862C95010136E4A7E9
:102EF000BC010000142F000800000020A00000000A
:102F0000D42B0008B42F0008A0000020605F000050
:102F1000E42B00080000000000000000000000009A
:102F2000D1D1E0D000000000D2D2000000000000AB
:102F30000000000000000000000000000000000091
:102F40000000000000000000000000000000000081
:102F50000000000000313233343536373839313231
:102F600033343536373839000000000000000000E7
:102F70000000000000313233343536373839313211
:102F800033343536373839000000000000000000C7
:102F90000000000000000000000000000000000031
:102FA00001020304010203040607080902040608DB
:042FB000000000001D
:0400000508000131BD
:00000001FF
